:0A0000002EC0FECFFDCFFCCFFBCFDA
:10000A00FACFF9CFF8CFF7CF54C0F5CFF4CFF3CF6B
:10001A00F2CFF1CFF0CFEFCFEECFEDCF1027E8033D
:10002A0064000A0001000010000110000100020033
:10003A00881300005700580059005A0041410042F5
:10004A00420043430000010002003800040004009B
:10005A003A000000F894EE27ECBBF1E0FBBFEBBFDF
:10006A00E5BFF8E1F1BDE1BD8DE0A2E0BB27ED936C
:10007A008A95E9F780E094E0A0E6ED930197E9F725
:10008A00E0E5F0E085919591009761F0A591B59131
:10009A0005901590BF01F00105900D920197E1F7C7
:1000AA00FB01F0CFEFE5EDBFE4E0EEBFC0E6D1E043
:1000BA001EC0EA93EFB7EA93E9EDE2BF20FE04C05F
:1000CA00E89420F8949805C020FC03C0689420F8AE
:1000DA00949AE991EFBFE9911895C4D1E8E8F3E160
:1000EA002F01689421F8E4E6F0E03F010895EFEF6C
:1000FA00E8BBE0E0E7BBEFEFE5BBE0E0E4BBE2BB77
:10010A00E0E1E1BBE1E0E3BFE0E1E2BFE0E0EFBD57
:10011A00EEBDEDBDECBDE7BDE6BDEBBDEABDE9BD9B
:10012A00E8BDE2BDE5BDE4BDE3BDE5BFE1E0E9BF91
:10013A00E0E0EBB9E8E0EAB9E6E8E0BDE0E0E0BD1E
:10014A00E7E6E9B9E0E8E8B9E0E0E0BF7894042C32
:10015A00052821F0F20131972F010AC0042C052845
:10016A0011F421FC01C004C079D1E89421F87ED1B0
:10017A00062C072821F0F30131973F0122C0062CF3
:10018A00072811F421FC01C01CC0989903C0E6E4B9
:10019A00F0E009C0999903C0E9E4F0E004C09A9933
:1001AA0008C0ECE4F0E0FA93EA9380E035D12296B5
:1001BA0094DF989B04C0999B02C09A9902C074D19B
:1001CA00F8CF72D1C4CFFFCF5D9BFECFE881ECB9E7
:1001DA0021960895EA81EA93F7DFA881B981ED9122
:1001EA00FD913196FE93EE93239608952697AAD110
:1001FA0010E0AC85BD85E0E0F0E0ED93FC93EA8980
:10020A00FB893196EA8BFB8B3197E4912E2FE030F4
:10021A0009F4FCC0E12FE03031F4253211F411E089
:10022A0001C047D1F2C0E130A1F4253211F441D125
:10023A00EBC012E040E000E02D3211F401E0E5C02D
:10024A002B3211F44BE2E1C0203211F440E2DDC05E
:10025A0002C0E23039F450E013E0203311F40068B0
:10026A00D4C003C0E33009F0D0C0203310F02A33E1
:10027A0008F007C0AAE05A9F502DE22FE0535E0F04
:10028A00C4C0E22FE33639F41DD11FD11BD1A4819A
:10029A00AA931FD1B9C0E33729F423D124D1EFD0CF
:1002AA001E2F07C0E03749F41CD11DD1F2D01E2FF2
:1002BA00086002600F7730E02DC0E43611F0E936AD
:1002CA0011F4046002C0E53729F4E6E2F0E014D143
:1002DA0015E00BC0E83511F4086003C0E83709F0EF
:1002EA0093C0E0E3F0E008D114E002FF11C0F9D0B6
:1002FA0006D1AB85AA2332F4EA85FB8517D1EA87B2
:10030A00FB874DE2403011F01F5F01C00B7F02C036
:10031A00E8D0F5D000FD10C0151770F407FF08C02B
:10032A0002FF04C00B7F242F115001C020E301C03B
:10033A0020E2BFD05150F0CF312F01FF15C030302D
:10034A0091F003FF05C0EE81FF812591D5D005C04C
:10035A00AE81BF812D91AE83BF83ABD0503009F0FF
:10036A0051503150ECCF47C020E3EE81FF81E6D0F7
:10037A00E887F987EE81FF813296BED0E885F98554
:10038A00AA85BB85AE17BF0750F02F5FA885B98530
:10039A00EA85FB85EA1BFB0BEA87FB87EFCF2A334B
:1003AA0028F003FF02C0295F01C0295D04FD19C0BE
:1003BA00213320F4A885B985119709F409C0531788
:1003CA0010F000FF01C011C020E207FF0AC020E3BD
:1003DA00006102FF06C00B7F4A937BD0503009F0C0
:1003EA00515067D0503009F051503150A885B98525
:1003FA00129708F0B9CF00FF07C0503029F05150CA
:10040A00E0E2EA9366D0F9CF10E0F9CEAC85BD857B
:10041A0091D09FD064960895FF92F82E269796D091
:10042A00DE0114967FD08D01E0E0EC83ED83EE834C
:10043A00EF83DE01189676D07DD0FA93EA931A9369
:10044A000A93EFEEF0E0FA93EA93FE013896FA93F4
:10045A00EA93CCDE82D02896FF900895E5B7E0684B
:10046A00E5BF0895E5B7EF77E5BF0895E5B7EF78FB
:10047A00E062E5BFEFB778948895EFBF0895A99138
:10048A00B991EE27FF276D91662311F03196FBCFC4
:10049A000895AA27BB27E991F9910590002011F048
:1004AA001196FBCFFD010895E1E0F0E0FA93EA939B
:1004BA002DC02A93ED85FE85FA93EA93E989FA8994
:1004CA0009950895E889F98908953497E88BF98B95
:1004DA000895ED85FE85FA93EA93E989FA890995E3
:1004EA000895F0DFF2CFA889B989149623D0EE8354
:1004FA00FF83FA93EA930895EE83FF830895A88908
:10050A00B989149617D0EA87FB870895E991F9917A
:10051A00309639F088EE93E00197F1F7A895319774
:10052A00C9F708950024AF0DB01D0895F195E1951E
:10053A00F0400895ED91FC91119708950590F4917A
:10054A00E02D08955A934A933A932A931A930A9359
:10055A0008955D814C813B812A8119810881089522
:00000001FF
